Microchip MPLAB XC8 Compiler V2.41

Linker command line:

-W-3 \
  --edf=E:/Program Files/Microchip/MPLABX/v6.15/packs/Microchip/PIC18F-Q_DFP/1.20.405/xc8\pic\dat\20230718171817_en.msgs \
  -pivt0x8=08h -cn -h+dist/default/debug\I2CPwm2.X.debug.sym \
  --cmf=dist/default/debug\I2CPwm2.X.debug.cmf -z -Q18F06Q40 \
  -oC:\Users\stephen\AppData\Local\Temp\xcAsqfc.\driver_tmp_3.o \
  --defsym=__MPLAB_BUILD=1 --fixupoverflow=error \
  -Mdist/default/debug/I2CPwm2.X.debug.map \
  --md=C:\Users\stephen\AppData\Local\Temp\xcAsqfc.\driver_tmp_0.dat -E1 \
  -ver=XC8 Compiler --acfsm=1493 -ACODE=00h-0FFFFh -ACONST=00h-0FFFFh \
  -ASMALLCONST=01600h-016FFhx234 -AMEDIUMCONST=01600h-0FFFFh \
  -ACOMRAM=0501h-055Fh -AABS1=0500h-014FFh -ABIGRAM=0501h-014FFh \
  -ARAM=0560h-05FFh,0600h-06FFhx15 -ABANK5=0560h-05FFh -ABANK6=0600h-06FFh \
  -ABANK7=0700h-07FFh -ABANK8=0800h-08FFh -ABANK9=0900h-09FFh \
  -ABANK10=0A00h-0AFFh -ABANK11=0B00h-0BFFh -ABANK12=0C00h-0CFFh \
  -ABANK13=0D00h-0DFFh -ABANK14=0E00h-0EFFh -ABANK15=0F00h-0FFFh \
  -ABANK16=01000h-010FFh -ABANK17=01100h-011FFh -ABANK18=01200h-012FFh \
  -ABANK19=01300h-013FFh -ABANK20=01400h-014FFh \
  -ASFR=00h-0FFhx4,0400h-045Fh,0460h-04FFh,01500h-015FFh \
  -ABIGSFR=00h-04FFh,01500h-015FFh -ACONFIG=0300000h-0300011h \
  -AIDLOC=0200000h-020003Fh -AEEDATA=0380000h-03801FFh -peeprom_data=EEDATA \
  -preset_vec=00h -ppowerup=CODE,init -pramtop=01600h \
  -psmallconst=SMALLCONST -pmediumconst=MEDIUMCONST -pconst=CONST \
  -AFARRAM=00h-00h \
  -prdata=COMRAM,nvrram=COMRAM,nvbit=COMRAM,rbss=COMRAM,rbit=COMRAM \
  -pfarbss=FARRAM,fardata=FARRAM,nvFARRAM=FARRAM \
  -pintsave_regs=BIGRAM,bigbss=BIGRAM,bigdata=BIGRAM -pbss=RAM \
  -pidata=CODE,irdata=CODE,ibigdata=CODE,ifardata=CODE -prparam=COMRAM \
  C:\Users\stephen\AppData\Local\Temp\xcAsqfc.\driver_tmp_9.o \
  dist/default/debug\I2CPwm2.X.debug.o 

Object code version is 3.11

Machine type is 18F06Q40



                Name                               Link     Load   Length Selector   Space Scale
C:\Users\stephen\AppData\Local\Temp\xcAsqfc.\driver_tmp_9.o
                config                           300000   300000        9        0       4
                init                                 1A       1A        4        4       0
                reset_vec                             0        0        4        0       0
dist/default/debug\I2CPwm2.X.debug.o
                config                           300000   300000        9        0       4
                ivt0x8                                8        8       12        4       0
                text65                              928      928        8        4       0
                text64                              920      920        8        4       0
                text63                              68A      68A       2E        4       0
                text62                              94E      94E        6        4       0
                text61                              918      918        8        4       0
                text60                              7C0      7C0       16        4       0
                text59                              7AA      7AA       16        4       0
                text58                              794      794       16        4       0
                text57                              77E      77E       16        4       0
                text56                              948      948        6        4       0
                text55                              910      910        8        4       0
                text54                              65C      65C       2E        4       0
                text53                              942      942        6        4       0
                text52                              820      820        E        4       0
                text51                              908      908        8        4       0
                text50                              900      900        8        4       0
                text49                              62E      62E       2E        4       0
                text48                              768      768       16        4       0
                text47                              23A      23A      132        4       0
                text46                              36C      36C       AC        4       0
                text45                              752      752       16        4       0
                text44                              93C      93C        6        4       0
                text43                              80E      80E       12        4       0
                text42                              7D6      7D6       14        4       0
                text41                              8F6      8F6        A        4       0
                text40                              8EC      8EC        A        4       0
                text39                              8E2      8E2        A        4       0
                text38                              8D8      8D8        A        4       0
                text37                              7FC      7FC       12        4       0
                text36                              7EA      7EA       12        4       0
                text35                              8CE      8CE        A        4       0
                text34                              8C4      8C4        A        4       0
                text33                              5D0      5D0       5E        4       0
                text32                              936      936        6        4       0
                text31                              930      930        6        4       0
                text30                              96C      96C        4        4       0
                text29                              968      968        4        4       0
                text28                              8BA      8BA        A        4       0
                text27                              8B0      8B0        A        4       0
                text26                              964      964        4        4       0
                text25                              960      960        4        4       0
                text24                              8A6      8A6        A        4       0
                text23                              89C      89C        A        4       0
                text22                              95C      95C        4        4       0
                text21                              958      958        4        4       0
                text20                              892      892        A        4       0
                text19                              888      888        A        4       0
                text18                              736      736       1C        4       0
                text17                              954      954        4        4       0
                text16                              71A      71A       1C        4       0
                text15                              562      562       6E        4       0
                text14                              6FE      6FE       1C        4       0
                text13                              87E      87E        A        4       0
                text12                              874      874        A        4       0
                text11                              86A      86A        A        4       0
                text10                              4F4      4F4       6E        4       0
                text9                               860      860        A        4       0
                text8                               856      856        A        4       0
                text7                               84C      84C        A        4       0
                text6                               486      486       6E        4       0
                text5                               842      842        A        4       0
                text4                               838      838        A        4       0
                text3                               82E      82E        A        4       0
                text2                               418      418       6E        4       0
                text1                               6DC      6DC       22        4       0
                text0                                1E       1E      21C        4       0
                cstackCOMRAM                        526      526       10      501       1
                bssCOMRAM                           501      501       13      501       1
                cinit                               6B8      6B8       24        4       0
                nvCOMRAM                            514      514       12      501       1

TOTAL           Name                               Link     Load   Length     Space
        CLASS   CODE           
                init                                 1A       1A        4         0
                reset_vec                             0        0        4         0
                ivt0x8                                8        8       12         0
                text65                              928      928        8         0
                text64                              920      920        8         0
                text63                              68A      68A       2E         0
                text62                              94E      94E        6         0
                text61                              918      918        8         0
                text60                              7C0      7C0       16         0
                text59                              7AA      7AA       16         0
                text58                              794      794       16         0
                text57                              77E      77E       16         0
                text56                              948      948        6         0
                text55                              910      910        8         0
                text54                              65C      65C       2E         0
                text53                              942      942        6         0
                text52                              820      820        E         0
                text51                              908      908        8         0
                text50                              900      900        8         0
                text49                              62E      62E       2E         0
                text48                              768      768       16         0
                text47                              23A      23A      132         0
                text46                              36C      36C       AC         0
                text45                              752      752       16         0
                text44                              93C      93C        6         0
                text43                              80E      80E       12         0
                text42                              7D6      7D6       14         0
                text41                              8F6      8F6        A         0
                text40                              8EC      8EC        A         0
                text39                              8E2      8E2        A         0
                text38                              8D8      8D8        A         0
                text37                              7FC      7FC       12         0
                text36                              7EA      7EA       12         0
                text35                              8CE      8CE        A         0
                text34                              8C4      8C4        A         0
                text33                              5D0      5D0       5E         0
                text32                              936      936        6         0
                text31                              930      930        6         0
                text30                              96C      96C        4         0
                text29                              968      968        4         0
                text28                              8BA      8BA        A         0
                text27                              8B0      8B0        A         0
                text26                              964      964        4         0
                text25                              960      960        4         0
                text24                              8A6      8A6        A         0
                text23                              89C      89C        A         0
                text22                              95C      95C        4         0
                text21                              958      958        4         0
                text20                              892      892        A         0
                text19                              888      888        A         0
                text18                              736      736       1C         0
                text17                              954      954        4         0
                text16                              71A      71A       1C         0
                text15                              562      562       6E         0
                text14                              6FE      6FE       1C         0
                text13                              87E      87E        A         0
                text12                              874      874        A         0
                text11                              86A      86A        A         0
                text10                              4F4      4F4       6E         0
                text9                               860      860        A         0
                text8                               856      856        A         0
                text7                               84C      84C        A         0
                text6                               486      486       6E         0
                text5                               842      842        A         0
                text4                               838      838        A         0
                text3                               82E      82E        A         0
                text2                               418      418       6E         0
                text1                               6DC      6DC       22         0
                text0                                1E       1E      21C         0
                cinit                               6B8      6B8       24         0

        CLASS   CONST          

        CLASS   SMALLCONST     

        CLASS   MEDIUMCONST    

        CLASS   COMRAM         
                cstackCOMRAM                        526      526       10         1
                bssCOMRAM                           501      501       13         1
                nvCOMRAM                            514      514       12         1

        CLASS   ABS1           

        CLASS   BIGRAM         

        CLASS   RAM            

        CLASS   BANK5          

        CLASS   BANK6          

        CLASS   BANK7          

        CLASS   BANK8          

        CLASS   BANK9          

        CLASS   BANK10         

        CLASS   BANK11         

        CLASS   BANK12         

        CLASS   BANK13         

        CLASS   BANK14         

        CLASS   BANK15         

        CLASS   BANK16         

        CLASS   BANK17         

        CLASS   BANK18         

        CLASS   BANK19         

        CLASS   BANK20         

        CLASS   SFR            

        CLASS   BIGSFR         

        CLASS   CONFIG         
                config                           300000   300000        9         4

        CLASS   IDLOC          

        CLASS   EEDATA         

        CLASS   FARRAM         

        CLASS   HEAP           

        CLASS   STACK          



SEGMENTS        Name                           Load    Length   Top    Selector   Space  Class

                reset_vec                      000000  000004  000004         0       0  CODE    
                ivt0x8                         000008  000968  000970         4       0  CODE    
                bssCOMRAM                      000501  000035  000536       501       1  COMRAM  


UNUSED ADDRESS RANGES

        Name                Unused          Largest block    Delta
        BANK10           000A00-000AFF              100
        BANK11           000B00-000BFF              100
        BANK12           000C00-000CFF              100
        BANK13           000D00-000DFF              100
        BANK14           000E00-000EFF              100
        BANK15           000F00-000FFF              100
        BANK16           001000-0010FF              100
        BANK17           001100-0011FF              100
        BANK18           001200-0012FF              100
        BANK19           001300-0013FF              100
        BANK20           001400-0014FF              100
        BANK5            000560-0005FF               A0
        BANK6            000600-0006FF              100
        BANK7            000700-0007FF              100
        BANK8            000800-0008FF              100
        BANK9            000900-0009FF              100
        BIGRAM           000536-0014FF              FCA
        BIGSFR           000000-0004FF              500
                         001500-0015FF              100
        CODE             000004-000007                4
                         000970-00FFFF             F690
        COMRAM           000536-00055F               2A
        CONFIG           300009-300011                9
        CONST            000004-000007                4
                         000970-00FFFF             F690
        EEDATA           380000-3801FF              200
        IDLOC            200000-20003F               40
        MEDIUMCONST      001600-00FFFF             EA00
        RAM              000560-0014FF              100
        SFR              000000-0004FF              100
                         001500-0015FF              100
        SMALLCONST       001600-00FFFF              100

                                  Symbol Table

I2C1_SlaveSendTxData@data                                     cstackCOMRAM 000526
I2C1_SlaveSetAddrIntHandler@handler                           cstackCOMRAM 00052B
I2C1_SlaveSetBusColIntHandler@handler                         cstackCOMRAM 00052B
I2C1_SlaveSetCounter@counter                                  cstackCOMRAM 000526
I2C1_SlaveSetIsrHandler@handler                               cstackCOMRAM 00052B
I2C1_SlaveSetReadIntHandler@handler                           cstackCOMRAM 00052B
I2C1_SlaveSetSlaveAddr@slaveAddr                              cstackCOMRAM 00052B
I2C1_SlaveSetSlaveMask@maskAddr                               cstackCOMRAM 00052B
I2C1_SlaveSetWrColIntHandler@handler                          cstackCOMRAM 00052B
I2C1_SlaveSetWriteIntHandler@handler                          cstackCOMRAM 00052B
IVTBASEH                                                      (abs)        00045E
IVTBASEL                                                      (abs)        00045D
IVTBASEU                                                      (abs)        00045F
PWM1_16BIT_Period_SetInterruptHandler@InterruptHandler        cstackCOMRAM 00052B
PWM1_16BIT_SetSlice1Output1DutyCycleRegister@registerValue    cstackCOMRAM 00052B
PWM1_16BIT_SetSlice1Output2DutyCycleRegister@registerValue    cstackCOMRAM 00052B
PWM1_16BIT_Slice1Output1_SetInterruptHandler@InterruptHandler cstackCOMRAM 00052B
PWM1_16BIT_Slice1Output2_SetInterruptHandler@InterruptHandler cstackCOMRAM 00052B
PWM2_16BIT_Period_SetInterruptHandler@InterruptHandler        cstackCOMRAM 00052B
PWM2_16BIT_SetSlice1Output1DutyCycleRegister@registerValue    cstackCOMRAM 00052B
PWM2_16BIT_SetSlice1Output2DutyCycleRegister@registerValue    cstackCOMRAM 00052B
PWM2_16BIT_Slice1Output1_SetInterruptHandler@InterruptHandler cstackCOMRAM 00052B
PWM2_16BIT_Slice1Output2_SetInterruptHandler@InterruptHandler cstackCOMRAM 00052B
PWM3_16BIT_Period_SetInterruptHandler@InterruptHandler        cstackCOMRAM 00052B
PWM3_16BIT_SetSlice1Output1DutyCycleRegister@registerValue    cstackCOMRAM 00052B
PWM3_16BIT_SetSlice1Output2DutyCycleRegister@registerValue    cstackCOMRAM 00052B
PWM3_16BIT_Slice1Output1_SetInterruptHandler@InterruptHandler cstackCOMRAM 00052B
PWM3_16BIT_Slice1Output2_SetInterruptHandler@InterruptHandler cstackCOMRAM 00052B
_ACTCON                                                       (abs)        0000AC
_ANSELA                                                       (abs)        000400
_ANSELC                                                       (abs)        000410
_I2C1ADB0                                                     (abs)        00028E
_I2C1ADR0                                                     (abs)        000290
_I2C1ADR1                                                     (abs)        000291
_I2C1ADR2                                                     (abs)        000292
_I2C1ADR3                                                     (abs)        000293
_I2C1BAUD                                                     (abs)        00029D
_I2C1CNTH                                                     (abs)        00028D
_I2C1CNTL                                                     (abs)        00028C
_I2C1CON0                                                     (abs)        000294
_I2C1CON0bits                                                 (abs)        000294
_I2C1CON1                                                     (abs)        000295
_I2C1CON1bits                                                 (abs)        000295
_I2C1CON2                                                     (abs)        000296
_I2C1ERRbits                                                  (abs)        000297
_I2C1PIEbits                                                  (abs)        00029B
_I2C1PIR                                                      (abs)        00029A
_I2C1PIRbits                                                  (abs)        00029A
_I2C1RXB                                                      (abs)        00028A
_I2C1SCLPPS                                                   (abs)        000271
_I2C1SDAPPS                                                   (abs)        000270
_I2C1STAT0bits                                                (abs)        000298
_I2C1STAT1bits                                                (abs)        000299
_I2C1TXB                                                      (abs)        00028B
_I2C1_Initialize                                              text18       000736
_I2C1_InterruptHandler                                        bssCOMRAM    00050E
_I2C1_IsRead                                                  text44       00093C
_I2C1_Isr                                                     text47       00023A
_I2C1_Open                                                    text33       0005D0
_I2C1_Read                                                    text31       000930
_I2C1_SlaveAddrCallBack                                       text63       00068A
_I2C1_SlaveAddrInterruptHandler                               bssCOMRAM    000508
_I2C1_SlaveBusColInterruptHandler                             bssCOMRAM    000506
_I2C1_SlaveClearBuff                                          text62       00094E
_I2C1_SlaveClearIrq                                           text61       000918
_I2C1_SlaveDefAddrInterruptHandler                            text64       000920
_I2C1_SlaveDefBusColInterruptHandler                          (abs)        000000
_I2C1_SlaveDefRdInterruptHandler                              text55       000910
_I2C1_SlaveDefWrColInterruptHandler                           (abs)        000000
_I2C1_SlaveDefWrInterruptHandler                              text50       000900
_I2C1_SlaveEnableIrq                                          text43       00080E
_I2C1_SlaveGetAddr                                            text65       000928
_I2C1_SlaveGetRxData                                          text32       000936
_I2C1_SlaveIsAddr                                             text60       0007C0
_I2C1_SlaveIsRead                                             text45       000752
_I2C1_SlaveIsRxBufFull                                        text59       0007AA
_I2C1_SlaveIsStop                                             text58       000794
_I2C1_SlaveIsTxBufEmpty                                       text57       00077E
_I2C1_SlaveOpen                                               text42       0007D6
_I2C1_SlaveRdCallBack                                         text54       00065C
_I2C1_SlaveRdInterruptHandler                                 bssCOMRAM    00050C
_I2C1_SlaveReleaseClock                                       text53       000942
_I2C1_SlaveSendTxData                                         text51       000908
_I2C1_SlaveSetAddrIntHandler                                  text41       0008F6
_I2C1_SlaveSetBusColIntHandler                                text40       0008EC
_I2C1_SlaveSetCounter                                         text52       000820
_I2C1_SlaveSetIsrHandler                                      text39       0008E2
_I2C1_SlaveSetReadIntHandler                                  text38       0008D8
_I2C1_SlaveSetSlaveAddr                                       text37       0007FC
_I2C1_SlaveSetSlaveMask                                       text36       0007EA
_I2C1_SlaveSetWrColIntHandler                                 text35       0008CE
_I2C1_SlaveSetWriteIntHandler                                 text34       0008C4
_I2C1_SlaveWrCallBack                                         text49       00062E
_I2C1_SlaveWrColInterruptHandler                              bssCOMRAM    000504
_I2C1_SlaveWrInterruptHandler                                 bssCOMRAM    00050A
_INLVLA                                                       (abs)        000404
_INLVLC                                                       (abs)        000414
_INTCON0bits                                                  (abs)        0004D6
_INTERRUPT_Initialize                                         text17       000954
_INTERRUPT_InterruptManager                                   text46       00036C
_LATA                                                         (abs)        0004BE
_LATC                                                         (abs)        0004C0
_ODCONA                                                       (abs)        000402
_ODCONC                                                       (abs)        000412
_OSCCON1                                                      (abs)        0000AD
_OSCCON3                                                      (abs)        0000AF
_OSCEN                                                        (abs)        0000B3
_OSCFRQ                                                       (abs)        0000B1
_OSCILLATOR_Initialize                                        text16       00071A
_OSCTUNE                                                      (abs)        0000B0
_PIE4bits                                                     (abs)        0004AC
_PIE5bits                                                     (abs)        0004AD
_PIE7bits                                                     (abs)        0004AF
_PIN_MANAGER_Initialize                                       text15       000562
_PIR4bits                                                     (abs)        0004B7
_PIR5bits                                                     (abs)        0004B8
_PIR7bits                                                     (abs)        0004BA
_PMD0                                                         (abs)        000063
_PMD1                                                         (abs)        000064
_PMD2                                                         (abs)        000065
_PMD3                                                         (abs)        000066
_PMD4                                                         (abs)        000067
_PMD5                                                         (abs)        000068
_PMD_Initialize                                               text14       0006FE
_PWM1CLK                                                      (abs)        000461
_PWM1CON                                                      (abs)        000469
_PWM1CONbits                                                  (abs)        000469
_PWM1CPRE                                                     (abs)        000465
_PWM1ERS                                                      (abs)        000460
_PWM1GIE                                                      (abs)        000468
_PWM1GIEbits                                                  (abs)        000468
_PWM1GIR                                                      (abs)        000467
_PWM1GIRbits                                                  (abs)        000467
_PWM1LDS                                                      (abs)        000462
_PWM1PIPOS                                                    (abs)        000466
_PWM1PRH                                                      (abs)        000464
_PWM1PRL                                                      (abs)        000463
_PWM1S1CFG                                                    (abs)        00046A
_PWM1S1P1H                                                    (abs)        00046C
_PWM1S1P1L                                                    (abs)        00046B
_PWM1S1P2H                                                    (abs)        00046E
_PWM1S1P2L                                                    (abs)        00046D
_PWM1_16BIT_Disable                                           text30       00096C
_PWM1_16BIT_Enable                                            text29       000968
_PWM1_16BIT_Initialize                                        text10       0004F4
_PWM1_16BIT_Period_DefaultInterruptHandler                    (abs)        000000
_PWM1_16BIT_Period_InterruptHandler                           nvCOMRAM     000514
_PWM1_16BIT_Period_SetInterruptHandler                        text13       00087E
_PWM1_16BIT_SetSlice1Output1DutyCycleRegister                 text28       0008BA
_PWM1_16BIT_SetSlice1Output2DutyCycleRegister                 text27       0008B0
_PWM1_16BIT_Slice1Output1_DefaultInterruptHandler             (abs)        000000
_PWM1_16BIT_Slice1Output1_InterruptHandler                    nvCOMRAM     000518
_PWM1_16BIT_Slice1Output1_SetInterruptHandler                 text12       000874
_PWM1_16BIT_Slice1Output2_DefaultInterruptHandler             (abs)        000000
_PWM1_16BIT_Slice1Output2_InterruptHandler                    nvCOMRAM     000516
_PWM1_16BIT_Slice1Output2_SetInterruptHandler                 text11       00086A
_PWM2CLK                                                      (abs)        000470
_PWM2CON                                                      (abs)        000478
_PWM2CONbits                                                  (abs)        000478
_PWM2CPRE                                                     (abs)        000474
_PWM2ERS                                                      (abs)        00046F
_PWM2GIE                                                      (abs)        000477
_PWM2GIEbits                                                  (abs)        000477
_PWM2GIR                                                      (abs)        000476
_PWM2GIRbits                                                  (abs)        000476
_PWM2LDS                                                      (abs)        000471
_PWM2PIPOS                                                    (abs)        000475
_PWM2PRH                                                      (abs)        000473
_PWM2PRL                                                      (abs)        000472
_PWM2S1CFG                                                    (abs)        000479
_PWM2S1P1H                                                    (abs)        00047B
_PWM2S1P1L                                                    (abs)        00047A
_PWM2S1P2H                                                    (abs)        00047D
_PWM2S1P2L                                                    (abs)        00047C
_PWM2_16BIT_Disable                                           text26       000964
_PWM2_16BIT_Enable                                            text25       000960
_PWM2_16BIT_Initialize                                        text6        000486
_PWM2_16BIT_Period_DefaultInterruptHandler                    (abs)        000000
_PWM2_16BIT_Period_InterruptHandler                           nvCOMRAM     00051A
_PWM2_16BIT_Period_SetInterruptHandler                        text9        000860
_PWM2_16BIT_SetSlice1Output1DutyCycleRegister                 text24       0008A6
_PWM2_16BIT_SetSlice1Output2DutyCycleRegister                 text23       00089C
_PWM2_16BIT_Slice1Output1_DefaultInterruptHandler             (abs)        000000
_PWM2_16BIT_Slice1Output1_InterruptHandler                    nvCOMRAM     00051E
_PWM2_16BIT_Slice1Output1_SetInterruptHandler                 text8        000856
_PWM2_16BIT_Slice1Output2_DefaultInterruptHandler             (abs)        000000
_PWM2_16BIT_Slice1Output2_InterruptHandler                    nvCOMRAM     00051C
_PWM2_16BIT_Slice1Output2_SetInterruptHandler                 text7        00084C
_PWM3CLK                                                      (abs)        00047F
_PWM3CON                                                      (abs)        000487
_PWM3CONbits                                                  (abs)        000487
_PWM3CPRE                                                     (abs)        000483
_PWM3ERS                                                      (abs)        00047E
_PWM3GIE                                                      (abs)        000486
_PWM3GIEbits                                                  (abs)        000486
_PWM3GIR                                                      (abs)        000485
_PWM3GIRbits                                                  (abs)        000485
_PWM3LDS                                                      (abs)        000480
_PWM3PIPOS                                                    (abs)        000484
_PWM3PRH                                                      (abs)        000482
_PWM3PRL                                                      (abs)        000481
_PWM3S1CFG                                                    (abs)        000488
_PWM3S1P1H                                                    (abs)        00048A
_PWM3S1P1L                                                    (abs)        000489
_PWM3S1P2H                                                    (abs)        00048C
_PWM3S1P2L                                                    (abs)        00048B
_PWM3_16BIT_Disable                                           text22       00095C
_PWM3_16BIT_Enable                                            text21       000958
_PWM3_16BIT_Initialize                                        text2        000418
_PWM3_16BIT_Period_DefaultInterruptHandler                    (abs)        000000
_PWM3_16BIT_Period_InterruptHandler                           nvCOMRAM     000520
_PWM3_16BIT_Period_SetInterruptHandler                        text5        000842
_PWM3_16BIT_SetSlice1Output1DutyCycleRegister                 text20       000892
_PWM3_16BIT_SetSlice1Output2DutyCycleRegister                 text19       000888
_PWM3_16BIT_Slice1Output1_DefaultInterruptHandler             (abs)        000000
_PWM3_16BIT_Slice1Output1_InterruptHandler                    nvCOMRAM     000524
_PWM3_16BIT_Slice1Output1_SetInterruptHandler                 text4        000838
_PWM3_16BIT_Slice1Output2_DefaultInterruptHandler             (abs)        000000
_PWM3_16BIT_Slice1Output2_InterruptHandler                    nvCOMRAM     000522
_PWM3_16BIT_Slice1Output2_SetInterruptHandler                 text3        00082E
_PWMIN0PPS                                                    (abs)        000257
_PWMIN1PPS                                                    (abs)        000258
_RA0PPS                                                       (abs)        000201
_RA1PPS                                                       (abs)        000202
_RC0PPS                                                       (abs)        000211
_RC1PPS                                                       (abs)        000212
_RC2PPS                                                       (abs)        000213
_RC3PPS                                                       (abs)        000214
_RC4PPS                                                       (abs)        000215
_RC5PPS                                                       (abs)        000216
_SLRCONA                                                      (abs)        000403
_SLRCONC                                                      (abs)        000413
_SYSTEM_Initialize                                            text1        0006DC
_TRISA                                                        (abs)        0004C6
_TRISC                                                        (abs)        0004C8
_WPUA                                                         (abs)        000401
_WPUC                                                         (abs)        000411
__HRAM                                                        (abs)        000000
__H__absolute__                                               __absolute__ 000000
__Habs1                                                       abs1         000000
__Hbank10                                                     bank10       000000
__Hbank11                                                     bank11       000000
__Hbank12                                                     bank12       000000
__Hbank13                                                     bank13       000000
__Hbank14                                                     bank14       000000
__Hbank15                                                     bank15       000000
__Hbank16                                                     bank16       000000
__Hbank17                                                     bank17       000000
__Hbank18                                                     bank18       000000
__Hbank19                                                     bank19       000000
__Hbank20                                                     bank20       000000
__Hbank5                                                      bank5        000000
__Hbank6                                                      bank6        000000
__Hbank7                                                      bank7        000000
__Hbank8                                                      bank8        000000
__Hbank9                                                      bank9        000000
__Hbigbss                                                     bigbss       000000
__Hbigdata                                                    bigdata      000000
__Hbigram                                                     bigram       000000
__Hbigsfr                                                     bigsfr       000000
__Hbss                                                        bss          000000
__HbssCOMRAM                                                  bssCOMRAM    000000
__Hcinit                                                      cinit        000000
__Hclrtext                                                    clrtext      000000
__Hcomram                                                     comram       000000
__Hconfig                                                     config       300009
__Hconst                                                      const        000000
__HcstackCOMRAM                                               cstackCOMRAM 000000
__Hdata                                                       data         000000
__Heeprom_data                                                eeprom_data  000000
__Hfarbss                                                     farbss       000000
__Hfardata                                                    fardata      000000
__Hheap                                                       heap         000000
__Hibigdata                                                   ibigdata     000000
__Hidata                                                      idata        000000
__Hidloc                                                      idloc        000000
__Hifardata                                                   ifardata     000000
__Hinit                                                       init         00001E
__Hintsave_regs                                               intsave_regs 000000
__Hirdata                                                     irdata       000000
__Hivt0x8                                                     ivt0x8       00001A
__Hmediumconst                                                mediumconst  000000
__HnvCOMRAM                                                   nvCOMRAM     000000
__HnvFARRAM                                                   nvFARRAM     000000
__Hnvbit                                                      nvbit        000000
__Hnvrram                                                     nvrram       000000
__Hparam                                                      rparam       000000
__Hpowerup                                                    powerup      000000
__Hram                                                        ram          000000
__Hramtop                                                     ramtop       001600
__Hrbit                                                       rbit         000000
__Hrbss                                                       rbss         000000
__Hrdata                                                      rdata        000000
__Hreset_vec                                                  reset_vec    000004
__Hrparam                                                     rparam       000000
__Hsfr                                                        sfr          000000
__Hsmallconst                                                 smallconst   000000
__Hspace_0                                                    (abs)        001600
__Hspace_1                                                    (abs)        000536
__Hspace_2                                                    (abs)        000000
__Hspace_4                                                    (abs)        600009
__Hstack                                                      stack        000000
__Hstruct                                                     struct       000000
__Htemp                                                       temp         000000
__Htext                                                       text         000000
__Htext0                                                      text0        000000
__Htext1                                                      text1        000000
__Htext10                                                     text10       000000
__Htext11                                                     text11       000000
__Htext12                                                     text12       000000
__Htext13                                                     text13       000000
__Htext14                                                     text14       000000
__Htext15                                                     text15       000000
__Htext16                                                     text16       000000
__Htext17                                                     text17       000000
__Htext18                                                     text18       000000
__Htext19                                                     text19       000000
__Htext2                                                      text2        000000
__Htext20                                                     text20       000000
__Htext21                                                     text21       000000
__Htext22                                                     text22       000000
__Htext23                                                     text23       000000
__Htext24                                                     text24       000000
__Htext25                                                     text25       000000
__Htext26                                                     text26       000000
__Htext27                                                     text27       000000
__Htext28                                                     text28       000000
__Htext29                                                     text29       000000
__Htext3                                                      text3        000000
__Htext30                                                     text30       000000
__Htext31                                                     text31       000000
__Htext32                                                     text32       000000
__Htext33                                                     text33       000000
__Htext34                                                     text34       000000
__Htext35                                                     text35       000000
__Htext36                                                     text36       000000
__Htext37                                                     text37       000000
__Htext38                                                     text38       000000
__Htext39                                                     text39       000000
__Htext4                                                      text4        000000
__Htext40                                                     text40       000000
__Htext41                                                     text41       000000
__Htext42                                                     text42       000000
__Htext43                                                     text43       000000
__Htext44                                                     text44       000000
__Htext45                                                     text45       000000
__Htext46                                                     text46       000000
__Htext47                                                     text47       000000
__Htext48                                                     text48       000000
__Htext49                                                     text49       000000
__Htext5                                                      text5        000000
__Htext50                                                     text50       000000
__Htext51                                                     text51       000000
__Htext52                                                     text52       000000
__Htext53                                                     text53       000000
__Htext54                                                     text54       000000
__Htext55                                                     text55       000000
__Htext56                                                     text56       000000
__Htext57                                                     text57       000000
__Htext58                                                     text58       000000
__Htext59                                                     text59       000000
__Htext6                                                      text6        000000
__Htext60                                                     text60       000000
__Htext61                                                     text61       000000
__Htext62                                                     text62       000000
__Htext63                                                     text63       000000
__Htext64                                                     text64       000000
__Htext65                                                     text65       000000
__Htext66                                                     text66       000000
__Htext7                                                      text7        000000
__Htext8                                                      text8        000000
__Htext9                                                      text9        000000
__LRAM                                                        (abs)        000001
__L__absolute__                                               __absolute__ 000000
__Labs1                                                       abs1         000000
__Lbank10                                                     bank10       000000
__Lbank11                                                     bank11       000000
__Lbank12                                                     bank12       000000
__Lbank13                                                     bank13       000000
__Lbank14                                                     bank14       000000
__Lbank15                                                     bank15       000000
__Lbank16                                                     bank16       000000
__Lbank17                                                     bank17       000000
__Lbank18                                                     bank18       000000
__Lbank19                                                     bank19       000000
__Lbank20                                                     bank20       000000
__Lbank5                                                      bank5        000000
__Lbank6                                                      bank6        000000
__Lbank7                                                      bank7        000000
__Lbank8                                                      bank8        000000
__Lbank9                                                      bank9        000000
__Lbigbss                                                     bigbss       000000
__Lbigdata                                                    bigdata      000000
__Lbigram                                                     bigram       000000
__Lbigsfr                                                     bigsfr       000000
__Lbss                                                        bss          000000
__LbssCOMRAM                                                  bssCOMRAM    000000
__Lcinit                                                      cinit        000000
__Lclrtext                                                    clrtext      000000
__Lcomram                                                     comram       000000
__Lconfig                                                     config       000000
__Lconst                                                      const        000000
__LcstackCOMRAM                                               cstackCOMRAM 000000
__Ldata                                                       data         000000
__Leeprom_data                                                eeprom_data  000000
__Lfarbss                                                     farbss       000000
__Lfardata                                                    fardata      000000
__Lheap                                                       heap         000000
__Libigdata                                                   ibigdata     000000
__Lidata                                                      idata        000000
__Lidloc                                                      idloc        000000
__Lifardata                                                   ifardata     000000
__Linit                                                       init         00001A
__Lintsave_regs                                               intsave_regs 000000
__Lirdata                                                     irdata       000000
__Livt0x8                                                     ivt0x8       000008
__Lmediumconst                                                mediumconst  000000
__LnvCOMRAM                                                   nvCOMRAM     000000
__LnvFARRAM                                                   nvFARRAM     000000
__Lnvbit                                                      nvbit        000000
__Lnvrram                                                     nvrram       000000
__Lparam                                                      rparam       000000
__Lpowerup                                                    powerup      000000
__Lram                                                        ram          000000
__Lramtop                                                     ramtop       001600
__Lrbit                                                       rbit         000000
__Lrbss                                                       rbss         000000
__Lrdata                                                      rdata        000000
__Lreset_vec                                                  reset_vec    000000
__Lrparam                                                     rparam       000000
__Lsfr                                                        sfr          000000
__Lsmallconst                                                 smallconst   000000
__Lspace_0                                                    (abs)        000000
__Lspace_1                                                    (abs)        000000
__Lspace_2                                                    (abs)        000000
__Lspace_4                                                    (abs)        000000
__Lstack                                                      stack        000000
__Lstruct                                                     struct       000000
__Ltemp                                                       temp         000000
__Ltext                                                       text         000000
__Ltext0                                                      text0        000000
__Ltext1                                                      text1        000000
__Ltext10                                                     text10       000000
__Ltext11                                                     text11       000000
__Ltext12                                                     text12       000000
__Ltext13                                                     text13       000000
__Ltext14                                                     text14       000000
__Ltext15                                                     text15       000000
__Ltext16                                                     text16       000000
__Ltext17                                                     text17       000000
__Ltext18                                                     text18       000000
__Ltext19                                                     text19       000000
__Ltext2                                                      text2        000000
__Ltext20                                                     text20       000000
__Ltext21                                                     text21       000000
__Ltext22                                                     text22       000000
__Ltext23                                                     text23       000000
__Ltext24                                                     text24       000000
__Ltext25                                                     text25       000000
__Ltext26                                                     text26       000000
__Ltext27                                                     text27       000000
__Ltext28                                                     text28       000000
__Ltext29                                                     text29       000000
__Ltext3                                                      text3        000000
__Ltext30                                                     text30       000000
__Ltext31                                                     text31       000000
__Ltext32                                                     text32       000000
__Ltext33                                                     text33       000000
__Ltext34                                                     text34       000000
__Ltext35                                                     text35       000000
__Ltext36                                                     text36       000000
__Ltext37                                                     text37       000000
__Ltext38                                                     text38       000000
__Ltext39                                                     text39       000000
__Ltext4                                                      text4        000000
__Ltext40                                                     text40       000000
__Ltext41                                                     text41       000000
__Ltext42                                                     text42       000000
__Ltext43                                                     text43       000000
__Ltext44                                                     text44       000000
__Ltext45                                                     text45       000000
__Ltext46                                                     text46       000000
__Ltext47                                                     text47       000000
__Ltext48                                                     text48       000000
__Ltext49                                                     text49       000000
__Ltext5                                                      text5        000000
__Ltext50                                                     text50       000000
__Ltext51                                                     text51       000000
__Ltext52                                                     text52       000000
__Ltext53                                                     text53       000000
__Ltext54                                                     text54       000000
__Ltext55                                                     text55       000000
__Ltext56                                                     text56       000000
__Ltext57                                                     text57       000000
__Ltext58                                                     text58       000000
__Ltext59                                                     text59       000000
__Ltext6                                                      text6        000000
__Ltext60                                                     text60       000000
__Ltext61                                                     text61       000000
__Ltext62                                                     text62       000000
__Ltext63                                                     text63       000000
__Ltext64                                                     text64       000000
__Ltext65                                                     text65       000000
__Ltext66                                                     text66       000000
__Ltext7                                                      text7        000000
__Ltext8                                                      text8        000000
__Ltext9                                                      text9        000000
__S0                                                          (abs)        000970
__S1                                                          (abs)        000536
__S4                                                          (abs)        000000
__S5                                                          (abs)        000000
___heap_hi                                                    (abs)        000000
___heap_lo                                                    (abs)        000000
___inthi_sp                                                   stack        000000
___intlo_sp                                                   stack        000000
___param_bank                                                 (abs)        000000
___rparam_used                                                (abs)        000001
___sp                                                         stack        000000
__accesstop                                                   (abs)        000560
__activetblptr                                                (abs)        000002
__end_of_I2C1_Initialize                                      text18       000752
__end_of_I2C1_IsRead                                          text44       000942
__end_of_I2C1_Isr                                             text47       00036C
__end_of_I2C1_Open                                            text33       00062E
__end_of_I2C1_Read                                            text31       000936
__end_of_I2C1_SlaveAddrCallBack                               text63       0006B8
__end_of_I2C1_SlaveClearBuff                                  text62       000954
__end_of_I2C1_SlaveClearIrq                                   text61       000920
__end_of_I2C1_SlaveDefAddrInterruptHandler                    text64       000928
__end_of_I2C1_SlaveDefRdInterruptHandler                      text55       000918
__end_of_I2C1_SlaveDefWrInterruptHandler                      text50       000908
__end_of_I2C1_SlaveEnableIrq                                  text43       000820
__end_of_I2C1_SlaveGetAddr                                    text65       000930
__end_of_I2C1_SlaveGetRxData                                  text32       00093C
__end_of_I2C1_SlaveIsAddr                                     text60       0007D6
__end_of_I2C1_SlaveIsRead                                     text45       000768
__end_of_I2C1_SlaveIsRxBufFull                                text59       0007C0
__end_of_I2C1_SlaveIsStop                                     text58       0007AA
__end_of_I2C1_SlaveIsTxBufEmpty                               text57       000794
__end_of_I2C1_SlaveOpen                                       text42       0007EA
__end_of_I2C1_SlaveRdCallBack                                 text54       00068A
__end_of_I2C1_SlaveReleaseClock                               text53       000948
__end_of_I2C1_SlaveSendTxData                                 text51       000910
__end_of_I2C1_SlaveSetAddrIntHandler                          text41       000900
__end_of_I2C1_SlaveSetBusColIntHandler                        text40       0008F6
__end_of_I2C1_SlaveSetCounter                                 text52       00082E
__end_of_I2C1_SlaveSetIsrHandler                              text39       0008EC
__end_of_I2C1_SlaveSetReadIntHandler                          text38       0008E2
__end_of_I2C1_SlaveSetSlaveAddr                               text37       00080E
__end_of_I2C1_SlaveSetSlaveMask                               text36       0007FC
__end_of_I2C1_SlaveSetWrColIntHandler                         text35       0008D8
__end_of_I2C1_SlaveSetWriteIntHandler                         text34       0008CE
__end_of_I2C1_SlaveWrCallBack                                 text49       00065C
__end_of_INTERRUPT_Initialize                                 text17       000958
__end_of_INTERRUPT_InterruptManager                           text46       000418
__end_of_OSCILLATOR_Initialize                                text16       000736
__end_of_PIN_MANAGER_Initialize                               text15       0005D0
__end_of_PMD_Initialize                                       text14       00071A
__end_of_PWM1_16BIT_Disable                                   text30       000970
__end_of_PWM1_16BIT_Enable                                    text29       00096C
__end_of_PWM1_16BIT_Initialize                                text10       000562
__end_of_PWM1_16BIT_Period_SetInterruptHandler                text13       000888
__end_of_PWM1_16BIT_SetSlice1Output1DutyCycleRegister         text28       0008C4
__end_of_PWM1_16BIT_SetSlice1Output2DutyCycleRegister         text27       0008BA
__end_of_PWM1_16BIT_Slice1Output1_SetInterruptHandler         text12       00087E
__end_of_PWM1_16BIT_Slice1Output2_SetInterruptHandler         text11       000874
__end_of_PWM2_16BIT_Disable                                   text26       000968
__end_of_PWM2_16BIT_Enable                                    text25       000964
__end_of_PWM2_16BIT_Initialize                                text6        0004F4
__end_of_PWM2_16BIT_Period_SetInterruptHandler                text9        00086A
__end_of_PWM2_16BIT_SetSlice1Output1DutyCycleRegister         text24       0008B0
__end_of_PWM2_16BIT_SetSlice1Output2DutyCycleRegister         text23       0008A6
__end_of_PWM2_16BIT_Slice1Output1_SetInterruptHandler         text8        000860
__end_of_PWM2_16BIT_Slice1Output2_SetInterruptHandler         text7        000856
__end_of_PWM3_16BIT_Disable                                   text22       000960
__end_of_PWM3_16BIT_Enable                                    text21       00095C
__end_of_PWM3_16BIT_Initialize                                text2        000486
__end_of_PWM3_16BIT_Period_SetInterruptHandler                text5        00084C
__end_of_PWM3_16BIT_SetSlice1Output1DutyCycleRegister         text20       00089C
__end_of_PWM3_16BIT_SetSlice1Output2DutyCycleRegister         text19       000892
__end_of_PWM3_16BIT_Slice1Output1_SetInterruptHandler         text4        000842
__end_of_PWM3_16BIT_Slice1Output2_SetInterruptHandler         text3        000838
__end_of_SYSTEM_Initialize                                    text1        0006FE
__end_of__initialization                                      cinit        0006D2
__end_of_main                                                 text0        00023A
__end_ofi2_I2C1_SlaveGetRxData                                text56       00094E
__end_ofi2_I2C1_SlaveIsRead                                   text48       00077E
__initialization                                              cinit        0006B8
__mediumconst                                                 mediumconst  000000
__pbssCOMRAM                                                  bssCOMRAM    000501
__pcinit                                                      cinit        0006B8
__pcstackCOMRAM                                               cstackCOMRAM 000526
__pivt0x8                                                     ivt0x8       000008
__pnvCOMRAM                                                   nvCOMRAM     000514
__ptext0                                                      text0        00001E
__ptext1                                                      text1        0006DC
__ptext10                                                     text10       0004F4
__ptext11                                                     text11       00086A
__ptext12                                                     text12       000874
__ptext13                                                     text13       00087E
__ptext14                                                     text14       0006FE
__ptext15                                                     text15       000562
__ptext16                                                     text16       00071A
__ptext17                                                     text17       000954
__ptext18                                                     text18       000736
__ptext19                                                     text19       000888
__ptext2                                                      text2        000418
__ptext20                                                     text20       000892
__ptext21                                                     text21       000958
__ptext22                                                     text22       00095C
__ptext23                                                     text23       00089C
__ptext24                                                     text24       0008A6
__ptext25                                                     text25       000960
__ptext26                                                     text26       000964
__ptext27                                                     text27       0008B0
__ptext28                                                     text28       0008BA
__ptext29                                                     text29       000968
__ptext3                                                      text3        00082E
__ptext30                                                     text30       00096C
__ptext31                                                     text31       000930
__ptext32                                                     text32       000936
__ptext33                                                     text33       0005D0
__ptext34                                                     text34       0008C4
__ptext35                                                     text35       0008CE
__ptext36                                                     text36       0007EA
__ptext37                                                     text37       0007FC
__ptext38                                                     text38       0008D8
__ptext39                                                     text39       0008E2
__ptext4                                                      text4        000838
__ptext40                                                     text40       0008EC
__ptext41                                                     text41       0008F6
__ptext42                                                     text42       0007D6
__ptext43                                                     text43       00080E
__ptext44                                                     text44       00093C
__ptext45                                                     text45       000752
__ptext46                                                     text46       00036C
__ptext47                                                     text47       00023A
__ptext48                                                     text48       000768
__ptext49                                                     text49       00062E
__ptext5                                                      text5        000842
__ptext50                                                     text50       000900
__ptext51                                                     text51       000908
__ptext52                                                     text52       000820
__ptext53                                                     text53       000942
__ptext54                                                     text54       00065C
__ptext55                                                     text55       000910
__ptext56                                                     text56       000948
__ptext57                                                     text57       00077E
__ptext58                                                     text58       000794
__ptext59                                                     text59       0007AA
__ptext6                                                      text6        000486
__ptext60                                                     text60       0007C0
__ptext61                                                     text61       000918
__ptext62                                                     text62       00094E
__ptext63                                                     text63       00068A
__ptext64                                                     text64       000920
__ptext65                                                     text65       000928
__ptext66                                                     text66       000000
__ptext7                                                      text7        00084C
__ptext8                                                      text8        000856
__ptext9                                                      text9        000860
__ramtop                                                      ramtop       001600
__smallconst                                                  smallconst   000000
_i2c1RdData                                                   bssCOMRAM    000512
_i2c1SlaveAddr                                                bssCOMRAM    000511
_i2c1SlaveState                                               bssCOMRAM    000510
_i2c1WrData                                                   bssCOMRAM    000513
_main                                                         text0        00001E
end_of_initialization                                         cinit        0006D2
i2_I2C1_SlaveGetRxData                                        text56       000948
i2_I2C1_SlaveIsRead                                           text48       000768
intlevel0                                                     text         000000
intlevel1                                                     text         000000
intlevel2                                                     text         000000
intlevel3                                                     text         000000
isa$std                                                       (abs)        000001
isa$xinst                                                     (abs)        000000
ivt0x8_base                                                   ivt0x8       000008
main@i                                                        cstackCOMRAM 00052F
main@pwmval                                                   cstackCOMRAM 000531
main@readin                                                   cstackCOMRAM 000533
stackhi                                                       (abs)        000000
stacklo                                                       (abs)        000000
start                                                         init         00001A
start_initialization                                          cinit        0006B8


MODULE INFORMATION

Module		Function		Class		Link	Load	Size
mcc_generated_files/pwm2_16bit.c
		_PWM2_16BIT_Disable		CODE           	0964	0000	4
		_PWM2_16BIT_Period_SetInterruptHandler		CODE           	0860	0000	10
		_PWM2_16BIT_Slice1Output1_SetInterruptHandler		CODE           	0856	0000	10
		_PWM2_16BIT_Slice1Output2_SetInterruptHandler		CODE           	084C	0000	10
		_PWM2_16BIT_Initialize		CODE           	0486	0000	110
		_PWM2_16BIT_SetSlice1Output1DutyCycleRegister		CODE           	08A6	0000	10
		_PWM2_16BIT_SetSlice1Output2DutyCycleRegister		CODE           	089C	0000	10
		_PWM2_16BIT_Enable		CODE           	0960	0000	4

mcc_generated_files/pwm2_16bit.c estimated size: 168

mcc_generated_files/interrupt_manager.c
		_INTERRUPT_Initialize		CODE           	0954	0000	4
		_INTERRUPT_InterruptManager		CODE           	036C	0000	172

mcc_generated_files/interrupt_manager.c estimated size: 176

mcc_generated_files/pin_manager.c
		_PIN_MANAGER_Initialize		CODE           	0562	0000	110

mcc_generated_files/pin_manager.c estimated size: 110

mcc_generated_files/i2c1_slave.c
		_I2C1_Read     		CODE           	0930	0000	6
		_I2C1_SlaveSetReadIntHandler		CODE           	08D8	0000	10
		_I2C1_SlaveDefAddrInterruptHandler		CODE           	0920	0000	8
		_I2C1_SlaveSetCounter		CODE           	0820	0000	14
		_I2C1_SlaveSetAddrIntHandler		CODE           	08F6	0000	10
		_I2C1_SlaveIsRead		CODE           	0752	0000	22
		_I2C1_SlaveSetIsrHandler		CODE           	08E2	0000	10
		_I2C1_SlaveIsAddr		CODE           	07C0	0000	22
		_I2C1_SlaveIsStop		CODE           	0794	0000	22
		_I2C1_SlaveEnableIrq		CODE           	080E	0000	18
		_I2C1_SlaveDefRdInterruptHandler		CODE           	0910	0000	8
		_I2C1_SlaveDefWrInterruptHandler		CODE           	0900	0000	8
		_I2C1_SlaveGetAddr		CODE           	0928	0000	8
		_I2C1_SlaveOpen		CODE           	07D6	0000	20
		_I2C1_SlaveSendTxData		CODE           	0908	0000	8
		_I2C1_SlaveSetSlaveAddr		CODE           	07FC	0000	18
		_I2C1_SlaveRdCallBack		CODE           	065C	0000	46
		_I2C1_SlaveWrCallBack		CODE           	062E	0000	46
		_I2C1_Isr      		CODE           	023A	0000	306
		_I2C1_Open     		CODE           	05D0	0000	94
		_I2C1_IsRead   		CODE           	093C	0000	6
		_I2C1_SlaveAddrCallBack		CODE           	068A	0000	46
		_I2C1_Initialize		CODE           	0736	0000	28
		_I2C1_SlaveSetWrColIntHandler		CODE           	08CE	0000	10
		_I2C1_SlaveIsTxBufEmpty		CODE           	077E	0000	22
		_I2C1_SlaveIsRxBufFull		CODE           	07AA	0000	22
		_I2C1_SlaveClearIrq		CODE           	0918	0000	8
		_I2C1_SlaveGetRxData		CODE           	0936	0000	6
		_I2C1_SlaveSetWriteIntHandler		CODE           	08C4	0000	10
		_I2C1_SlaveSetBusColIntHandler		CODE           	08EC	0000	10
		_I2C1_SlaveReleaseClock		CODE           	0942	0000	6
		_I2C1_SlaveSetSlaveMask		CODE           	07EA	0000	18
		_I2C1_SlaveClearBuff		CODE           	094E	0000	6

mcc_generated_files/i2c1_slave.c estimated size: 902

mcc_generated_files/pwm1_16bit.c
		_PWM1_16BIT_Disable		CODE           	096C	0000	4
		_PWM1_16BIT_Period_SetInterruptHandler		CODE           	087E	0000	10
		_PWM1_16BIT_Slice1Output1_SetInterruptHandler		CODE           	0874	0000	10
		_PWM1_16BIT_Slice1Output2_SetInterruptHandler		CODE           	086A	0000	10
		_PWM1_16BIT_Initialize		CODE           	04F4	0000	110
		_PWM1_16BIT_SetSlice1Output1DutyCycleRegister		CODE           	08BA	0000	10
		_PWM1_16BIT_SetSlice1Output2DutyCycleRegister		CODE           	08B0	0000	10
		_PWM1_16BIT_Enable		CODE           	0968	0000	4

mcc_generated_files/pwm1_16bit.c estimated size: 168

shared
		i2_I2C1_SlaveIsRead		CODE           	0768	0000	22
		i2_I2C1_SlaveGetRxData		CODE           	0948	0000	6
		__initialization		CODE           	06B8	0000	26

shared estimated size: 54

mcc_generated_files/mcc.c
		_PMD_Initialize		CODE           	06FE	0000	28
		_OSCILLATOR_Initialize		CODE           	071A	0000	28
		_SYSTEM_Initialize		CODE           	06DC	0000	34

mcc_generated_files/mcc.c estimated size: 90

mcc_generated_files/pwm3_16bit.c
		_PWM3_16BIT_Enable		CODE           	0958	0000	4
		_PWM3_16BIT_Disable		CODE           	095C	0000	4
		_PWM3_16BIT_Period_SetInterruptHandler		CODE           	0842	0000	10
		_PWM3_16BIT_Slice1Output1_SetInterruptHandler		CODE           	0838	0000	10
		_PWM3_16BIT_Slice1Output2_SetInterruptHandler		CODE           	082E	0000	10
		_PWM3_16BIT_Initialize		CODE           	0418	0000	110
		_PWM3_16BIT_SetSlice1Output1DutyCycleRegister		CODE           	0892	0000	10
		_PWM3_16BIT_SetSlice1Output2DutyCycleRegister		CODE           	0888	0000	10

mcc_generated_files/pwm3_16bit.c estimated size: 168

main.c
		_main          		CODE           	001E	0000	540

main.c estimated size: 540

